:0300000002036296
:03004300020100B7
:1001000002013C000201580002011800020129000E
:10011000020120000201180032E591C2E4F59122AB
:10012000C0E0C2003119D0E032C0E0E5874401F5FB
:10013000870000003119D0E032C2DC32C0D0C0E00C
:10014000C082C08312016931197401907FABF0D075
:1001500083D082D0E0D0D032C0D0C0E0C082C08393
:090160001205FA3119740280E263
:10016900907FE8E0A2E79202545C7051E0A2E0823D
:10017900E1404A30E50274035403C4F540A3E05456
:100189000F45401201D52001343002182003209078
:100199007F027846754003E6F0158218D540F8E6E7
:1001A900907FB5F0754002907FB4E04540F022851C
:1001B9008240E583907FD4F0E540A380E675400353
:1001C90080E5E02582F58250020583229001FA310B
:1001D900CCE09001FA31CCC082C0837845E4F618AE
:1001E900F6187601907FEAE0F5F0A3E0C201C203B8
:1001F900226D404040404081406A74404040404048
:1002090040714040404040A540404040404040404F
:1002190040714240404040404040404040404040A2
:1002290040405663404040404040435D404040406C
:1002390040D201223000FA907FC5F0907FAAE054A5
:100249000160FBF00203CA3000E70876182230008B
:10025900E0F541223000DA08A641223000D50876BF
:100269000122760222E5F060061470C5D20022C28E
:100279000022D203149002C560B9149002D760B36A
:100289001470AE900316E5F0601EF54031CBE060C6
:10029900A0E5401480F2D203C394219002E960934F
:1002A900149002F9608D8089E0FFF5F07800F2087A
:0C02B900A3E0DFFAD0E0D0E0E5F021A9DE
:1002C500120101010000004042420001000101024B
:1002D5000001090222000101008032090400000129
:1002E50003000000092100010001221D000705810E
:1002F500034000640600FF0901A101190129021547
:100305000026FF007508952881021901290291022E
:10031500C0040309042C0355005300420020004487
:100325000065007300690067006E002000420079D7
:100335000020004500780061006D0070006C0065CC
:10034500001A035200650061006400650072002018
:100355000042006F0061007200640000007581EBCF
:1003650075927F78D6E254F3F21203B9E24406F2AD
:10037500E4F520F54678487F2B7408F608DFFC780D
:1003850093E4F2799CF4F37895799EE254F0F2E3E4
:10039500440FF37898E254F0F278ACF208F208745E
:1003A50003F2087401F278AA74FFF275E80175A8E2
:1003B500C00080FD75406490FB50A3E582458370C5
:1003C500F9D540F322758601907EC078497F07E014
:1003D50030E702743FC394205002743C75F005A4C5
:1003E500058690041A2582F582E5F03583F5837E2E
:1003F50005E0F6A308DEFA7600080586A3DFD0053A
:1004050086907E8078497F28E6F0A308DFFA907F02
:10041500B77428F022000000000000007D000000F5
:1004250070007000147F147F14122A7F2A246264DE
:1004350008132336495522050050600000001C2290
:1004450041000041221C0014083E081408083E081B
:100455000800050600000808080808000303000056
:1004650002040810203E4549513E00217F0100212C
:100475004345493142415169460C14247F04725168
:1004850051514E1E29494906404748506036494951
:1004950049363049494A3C0033330000006566005F
:1004A50000000814224114141414144122140800E5
:1004B500204045483026494F413E3F4848483F7F08
:1004C500494949363E414141227F4141221C7F49EC
:1004D5004949417F484848403E4149492F7F0808DE
:1004E500087F00417F41000201417E407F081422C0
:1004F500417F010101017F2018207F7F1008047FC3
:100505003E4141413E7F484848303E4145423D7F5E
:10051500484C4A31314949494640407F40407E0177
:1005250001017E7C0201027C7E010E017E631408BE
:10053500146370080708704345495161007F4141C4
:10054500007F4141417F0041417F00102040201044
:1005550001010101010040201000021515150F7F52
:100565000911110E0E111111020E1111097F0E152F
:1005750015150C083F484020182525253E7F0810F5
:10058500100F00115F01000201115E007F040A11C6
:100595000000417F01001F100C100F1F0810100FE5
:1005A5000E1111110E1F14141408081414141F1F12
:1005B500081010080915151502107E1101021E01FB
:1005C50001011F1C0201021C1E0106011E110A0465
:1005D5000A11180505051E111315191100083641D4
:1005E5000000007F0000004136080008082A1C08AA
:1005F500081C2A0808D54A37754A19789879967AD1
:1006050001E548B4271A907F9CE4F0740CF27999BF
:10061500E3F54779967410F274FFF07A0B7548FF8D
:10062500E4F3EAF2E4F20548E5482449F8E6F32262
:00000001FF
